:020000040000FA
:04000000E8303A2882
:040004000034003490
:08000800A000030EA100831209
:100010008B1C32288B1032181428B21C3228643002
:10002000010203183128182800001628172818285C
:1000300019281A281B281C281D281E281F283210A2
:10004000B214A810031005190314AA0DA90DA80DC8
:10005000B10B322832152A08AF002908AE00280853
:10006000AD00B21081010B11210E8300A00E200EF5
:02007000090085
:0C007400203084008001840A80300402E7
:10008000031C3C281230B100F42183160C30850586
:1000900087018312850187010730990000309A009B
:1000A000103083168E008312603083168F00831207
:1000B0000030831691009F008312C83083168100A0
:1000C000831231309000003083168C008312103080
:1000D0008B00482381018E018F010B118B100B10B7
:1000E0008C018B17812032199720B40B7F280310C5
:1000F00085190314BA0DF0303A0203194F21E52394
:1001000072286400321808000B1D08000B11B21091
:1001100032141230B100051D9228331483160113D6
:10012000831208003310831601178312080032115E
:100130000130B7008B132030370783169B001C1447
:100140001A088312A400A500C030A5061030370796
:1001500083169B001C141A088312A3000030370773
:1001600083169B001C141A088312A2008B17331CE1
:10017000BF2822090339A200A309A409A50922085E
:100180002D02031D492923082E02031D4929240895
:100190002F02031D492901303702031DD4283E18C0
:1001A000D4283E143F140F2202303702031DDD28ED
:1001B000BE18DD28BE143F14222203303702031D6F
:1001C000E6283E19E6283E153F1435220430370252
:1001D000031DEF28BE19EF28BE153F144822053035
:1001E0003702031DF8283E1AF8283E163F145B22FA
:1001F00006303702031D0129BE1A0129BE163F141D
:100200006E2207303702031D0A293E1B0A293E17BA
:100210003F14812208303702031D1329BE1B132906
:10022000BE173F148D2209303702031D1C295E18AA
:100230001C295E143F1499220A303702031D252918
:10024000DE182529DE143F14A7220B303702031DC8
:100250002E295E192E295E153F14B5220C30370267
:10026000031D3729DE193729DE153F14C3220D304F
:100270003702031D40295E1A40295E163F14D12221
:100280000E303702031D4929DE1A4929DE163F14B4
:10029000DE22B70A0F303702031808009A2801300F
:1002A000B600B400B500B70085018701B213812004
:1002B000B40B6729031085190314BA0DF0303A0204
:1002C00003198E29B50B67299630B5009821321D88
:1002D00057293211331C71292D090339AD00AE099C
:1002E000AF092F1CB2132F1C5729B21B57292E18E8
:1002F0005729B2178B1320303707BC002F08BB00DB
:10030000DF2110303707BC002E08BB00DF21003092
:100310003707BC002D08BB00DF218B178501870143
:10032000B70AB6010F303702031C572948230800CB
:100330000130370203190223023037020319072361
:100340000330370203190C23043037020319112339
:1003500005303702031916230630370203191B2311
:1003600007303702031920230830370203192523E9
:100370000930370203192A230A30370203192F23C1
:100380000B303702031934230C3037020319392399
:100390000D30370203193E230E3037020319432371
:1003A00008003F1C08003F101030BC003E08BB0096
:1003B000DF213030BC005E08BB00DF2108008B135A
:1003C0003B0883161C159A0083123C0883169B0079
:1003D00055309D00AA309D009C1464009C18ED29A6
:1003E0001C1183128B170800831610309B001C14FD
:1003F0001A088312BE00831630309B001C141A08A2
:100400008312DE00FF30C800CA15CB15CC15CD1500
:10041000CE15CF15D015D115D215D3150800C13082
:10042000BE05FF30DE055F1E1C2A1C30C405C0005F
:100430000030C200C6005F101C30D4000030D50070
:10044000922B0800C230BE05FF30DE055F1E2F2A4A
:100450003330C405C0000030C200C6005F10333026
:10046000D4000030D500922B0800C430BE05FF3008
:10047000DE055F1E422A3930C405C0000030C200CC
:10048000C6005F103930D4000030D500922B080030
:10049000C830BE05FF30DE05DF1E552A4C30C405CE
:1004A000C0000030C200C6005F104C30D6000030E3
:1004B000D7009D2B0800D030BE05FF30DE05DF1EC3
:1004C000682AC330C405C0000030C200C6005F10F7
:1004D000C330D6000030D7009D2B0800E030BE05A9
:1004E000FF30DE05DF1E7B2AC930C405C0000030A6
:1004F000C200C6005F10C930D6000030D7009D2B67
:1005000008007F30BE050030DE054030C505C10063
:100510000030C300C700EB2A0800BF30BE05003022
:10052000DE058030C505C1000030C300C700F62AD3
:1005300008003F30BE050130DE05A42A0030C505A5
:10054000C1000030C300C7005F15DF1508003F3051
:10055000BE050230DE05B22A0030C505C1000030FC
:10056000C300C7005F15DF1508003F30BE0504302B
:10057000DE05C02A0030C505C1000030C300C70039
:100580005F15DF1508003F30BE050830DE05CE2AB6
:100590000030C505C1000030C300C7005F15DF157E
:1005A00008003F30BE051030DE05DC2A0030C505EE
:1005B000C1000030C300C7005F1108003F30BE0516
:1005C0002030DE05E92A0030C505C1000030C30037
:1005D000C7005F1108005F1A08005F16DF12540899
:1005E000C405C0005508C200C6000800DF1A080094
:1005F000DF165F125608C405C0005708C200C600C7
:1006000008000800033085061230870608003030E5
:1006100085061630870608001230850616308706D4
:10062000080003308506093087060800303085064B
:100630002930870608001230850629308706080011
:100640000030850616308706080000308506293000
:100650008706080022308506003087060800213012
:1006600085060030870608002230850600308706A0
:1006700008002130850600308706080032308506E4
:1006800000308706080031308506003087060800F4
:10069000A8235F12DF12BE1BDF16DF1E5F163E1897
:1006A0000F22BE1822223E193522BE1948223E1AB8
:1006B0005B22BE1A6E223E1B8122BE1B8D225E185B
:1006C0009922DE18A7225E19B522DE19C3225E1A0E
:1006D000D122DE1ADE220800B601B401B5013D1CAC
:1006E000742BBD01BD14762BBD013D143D08B60031
:1006F00064007A2B7B2B7C2B7D2B7E2BFF30B51B54
:100700008500B51F8501B40B782BB50B782B031032
:10071000B60CB608031D782B0030BC003D08BB00AA
:10072000DF2108004030BC005408BB00DF215030FE
:10073000BC005508BB00DF2108006030BC00560833
:10074000BB00DF217030BC005708BB00DF21080070
:10075000831640309B001C141A088312D4008316A1
:1007600050309B001C141A088312D5008316603089
:100770009B001C141A088312D600831670309B004D
:100780001C141A088312D700080005125C180516FD
:10079000DC1C8512DC1885165C1D05105C1905141F
:1007A000DC1D8510DC1985145C1E87105C1A87140B
:1007B000DC1E0711DC1A07155C1F07105C1B0714F1
:1007C000DC1F8712DC1B871608008F08031908003E
:1007D0008F0178308E00C80F272EC80ADF19172C1A
:1007E000441C172C461C082CCA1CF92BCA014A159C
:1007F000252C4A1DFE2BCA01CA15252CCA1D032C07
:10080000CA014A16252C4A1E252CCA01CA14252CB9
:100810004A1D0D2CCA014A16252CCA1D122CCA01CC
:100820004A16252C4A1E252CCA01CA14252CCA1C7E
:100830001C2CCA014A15252C4A1D212CCA01CA1597
:10084000252C4A1E252CCA014A15DF194E2CC41C22
:100850004E2CC61C3F2CCB1C302CCB014B155C2CDA
:100860004B1D352CCB01CB155C2CCB1D3A2CCB0171
:100870004B165C2C4B1E5C2CCB01CB145C2C4B1D03
:10088000442CCB014B165C2CCB1D492CCB014B16B9
:100890005C2C4B1E5C2CCB01CB145C2CCB1C532C46
:1008A000CB014B155C2C4B1D582CCB01CB155C2C74
:1008B0004B1E5C2CCB014B15DF19852C441D852C60
:1008C000461D762CCC1C672CCC014C15932C4C1D52
:1008D0006C2CCC01CC15932CCC1D712CCC014C165E
:1008E000932C4C1E932CCC01CC14932C4C1D7B2CA4
:1008F000CC014C16932CCC1D802CCC014C16932C87
:100900004C1E932CCC01CC14932CCC1C8A2CCC01E7
:100910004C15932C4C1D8F2CCC01CC15932C4C1EBC
:10092000932CCC014C15DF19BD2CC41DBD2CC61D4C
:10093000AE2CCD1C9F2CCD014D155F13CB2C4D1D26
:10094000A42CCD01CD15CB2CCD1DA92CCD014D1640
:10095000CB2C4D1ECB2CCD01CD14CB2C4D1DB32C4F
:10096000CD014D16CB2CCD1DB82CCD014D16CB2C69
:100970004D1ECB2CCD01CD14CB2CCD1CC22CCD01CA
:100980004D15CB2C4D1DC72CCD01CD15CB2C4D1E9F
:10099000CB2CCD014D15DF19F62C5F1BF62C441E18
:1009A000F62C461EE72CCE1CD82CCE014E15042D5D
:1009B0004E1DDD2CCE01CE15042DCE1DE22CCE0118
:1009C0004E16042D4E1E042DCE01CE14042D4E1DA8
:1009D000EC2CCE014E16042DCE1DF12CCE014E1660
:1009E000042D4E1E042DCE01CE14042DCE1CFB2C46
:1009F000CE014E15042D4E1D002DCE01CE15042D19
:100A00004E1E042DCE014E15DF192D2DC41E2D2D89
:100A1000C61E1E2DCF1C0F2DCF014F153B2D4F1D78
:100A2000142DCF01CF153B2DCF1D192DCF014F1602
:100A30003B2D4F1E3B2DCF01CF143B2D4F1D232DA2
:100A4000CF014F163B2DCF1D282DCF014F163B2D2B
:100A50004F1E3B2DCF01CF143B2DCF1C322DCF018C
:100A60004F153B2D4F1D372DCF01CF153B2D4F1E61
:100A70003B2DCF014F15DF19642D441F642D461FF8
:100A8000552DD01C462DD0015015722D501D4B2DCB
:100A9000D001D015722DD01D502DD0015016722DC1
:100AA000501E722DD001D014722D501D5A2DD00120
:100AB0005016722DD01D5F2DD0015016722D501E74
:100AC000722DD001D014722DD01C692DD00150157B
:100AD000722D501D6E2DD001D015722D501E722D0D
:100AE000D0015015DF199B2DC41F9B2DC61F8C2DC7
:100AF000D11C7D2DD1015115A92D511D822DD10162
:100B0000D115A92DD11D872DD1015116A92D511E09
:100B1000A92DD101D114A92D511D912DD10151160D
:100B2000A92DD11D962DD1015116A92D511EA92DEA
:100B3000D101D114A92DD11CA02DD1015115A92D60
:100B4000511DA52DD101D115A92D511EA92DD101C0
:100B50005115DF19D32D451FD32D471FC42DD21C8E
:100B6000B52DD2015215DF13E12D521DBA2DD20140
:100B7000D215E12DD21DBF2DD2015216E12D521EEC
:100B8000E12DD201D214E12D521DC92DD2015216F0
:100B9000E12DD21DCE2DD2015216E12D521EE12D96
:100BA000D201D214E12DD21CD82DD2015215E12D43
:100BB000521DDD2DD201D215E12D521EE12DD201A3
:100BC0005215DF190C2EDF1B0C2EC51F0C2EC71F54
:100BD000FD2DD31CEE2DD30153151A2E531DF32DCD
:100BE000D301D3151A2ED31DF82DD30153161A2E67
:100BF000531E1A2ED301D3141A2E531D022ED301C5
:100C000053161A2ED31D072ED30153161A2E531E18
:100C10001A2ED301D3141A2ED31C112ED30153151F
:100C20001A2E531D162ED301D3151A2E531E1A2E0B
:100C3000D3015315D1214008C4004108C5005F18F5
:100C4000DF145F1CDF105F19DF155F1DDF1148081F
:100C5000C9000C304A05031D05120C304B05031D5D
:100C600085120C304C05031D05100C304D05031D7D
:100C700085100C304E05031D87100C304F05031DE9
:100C800007110C305005031D07100C305105031DD2
:100C900087120C305205031D07120C305305031D3B
:100CA000871149080E020318812E12304A05031DD0
:100CB000051612304B05031D851612304C05031D19
:100CC000051412304D05031D851412304E05031D09
:100CD000871412304F05031D071512305005031DF0
:100CE000071412305105031D871612305205031DDB
:100CF000071612305305031D8715FF3048020319EC
:100D000008008F08031D0800812049080E02031CFB
:100D1000812E18304A05031D051206304A05031DB1
:100D2000051618304B05031D851206304B05031DB3
:100D3000851618304C05031D051006304C05031DA3
:100D4000051418304D05031D851006304D05031D93
:100D5000851418304E05031D871006304E05031DFF
:100D6000871418304F05031D071106304F05031D6A
:100D7000071518305005031D071006305005031DD8
:100D8000071418305105031D871206305105031D45
:100D9000871618305205031D071206305205031D31
:100DA000071618305305031D871106305305031D20
:040DB000871508009B
:084000000D0003000600090099
:02400E00CC33B1
:10420000010003000300030003000200020002009B
:104210000200000000000000000003000300030093
:10422000420000000000000000000000000000004C
:104230000000C000C000C000C000C000C000C0003E
:10424000FF00C300F300CF00FF00C300F300CF0066
:10425000FF00C300F300CF00FF00C300F300CF0056
:104260000000FF00FF00FF00FF00FF00FF00FF0055
:10427000FF00FF00FF00FF00FF00FF00FF00FF0046
:1042800033000300FF00FF00FF00FF00FF00FF00FE
:10429000FF00FF00FF00FF00FF00FF00FF00FF0026
:1042A0000000C000FF00FF00FF00FF00FF00FF0054
:1042B000FF00FF00FF00FF00FF00FF00FF00FF0006
:1042C000C300FF00FF00FF00FF00FF00FF00FF0032
:1042D000FF00FF00FF00FF00FF00FF00FF00FF00E6
:1042E0000000FF00FF00FF00FF00FF00FF00FF00D5
:1042F000FF00FF00FF00FF00FF00FF00FF00AA001B
:00000001FF
